S02000002E2E5C62696E5C6F70656E626C745F73746D3332663230372E73726563AC
S31508000000008000202D1900087B1900087D190008BA
S315080000107F190008811900088319000800000000EC
S31508000020000000000000000000000000851900081C
S315080000308719000800000000891900088B190008B4
S315080000408F190008911900089319000895190008D6
S3150800005097190008991900089B1900089D190008A6
S315080000609F190008A1190008A3190008A519000876
S31508000070A7190008A9190008AB190008AD19000846
S31508000080AF190008B1190008B3190008B519000816
S31508000090B7190008B9190008BB190008BD190008E6
S315080000A0BF190008C1190008C3190008C5190008B6
S315080000B0C7190008C9190008CB190008CD19000886
S315080000C0CF190008D1190008D3190008D519000856
S315080000D0D7190008D9190008DB190008DD19000826
S315080000E0DF190008E1190008E3190008E5190008F6
S315080000F0E7190008E9190008EB190008ED190008C6
S31508000100EF190008F1190008F3190008F519000895
S31508000110F7190008F9190008FB190008FD19000865
S31508000120FF190008011A0008031A0008051A000832
S31508000130071A0008091A00080B1A00080D1A000801
S315080001400F1A0008111A0008131A0008151A0008D1
S31508000150171A0008191A00081B1A00081D1A0008A1
S315080001601F1A0008211A0008231A0008251A000871
S31508000170271A0008291A00082B1A00082D1A000841
S315080001802F1A000810B5054C237833B9044B13B160
S315080001900448AFF300800123237010BD84000020BB
S315080001A0000000007C510008084B10B51BB1084937
S315080001B00848AFF300800848036803B910BD074B29
S315080001C0002BFBD0BDE81040184700BF0000000018
S315080001D0880000207C5100088400002000000000F0
S315080001E0154B002B08BF134B9D46A3F5803A0021FB
S315080001F08B460F461348144A121A04F091FB0F4B0C
S31508000200002B00D098470E4B002B00D098470020B3
S31508000210002104000D000D48002802D00C48AFF359
S31508000220008004F057FB2000290000F0F5FF04F0D9
S315080002303DFB00BF00000800008000200000000011
S315080002400000000084000020EC0F002000000000E1
S315080002500000000008B500F0D5F84FF40051034837
S3150800026000F01CFE003018BF012008BD000802403F
S3150800027008B5642000F094F808BD00BF08B500F082
S3150800028095F808BD00B5C7B04FF48C7200216846D2
S3150800029004F046FB6946094804F008F840B9009B93
S315080002A043B19DF8080080F01000C0F3001002E08A
S315080002B0002000E0002047B05DF804FB4C49000828
S315080002C0004870474C49000808B50748002380F8DD
S315080002D028320A22054903F053FC18B90122024BB9
S315080002E083F8282208BD00BFA0000020684900083E
S315080002F070B50E4B93F82832012B02D10B4803F048
S315080003000BFF01F0DDFB00F16406094D402403E014
S3150800031001F0D6FB864205D32146284600F008FFA1
S315080003200028F5D0034803F0E7FF70BDA0000020C1
S31508000330004800404C49000808B5044B93F8283299
S31508000340012B02D1014803F0E7FE08BDA0000020FA
S3150800035070B50646104B93F82832012B0AD10E4980
S3150800036004F050F8002805DA0B48002380F82832F4
S3150800037003F0D2FE317871B1084C8025204600F092
S31508000380CFFE2946204600F0D3FE0028F9D016F8FD
S31508000390011F0029F2D170BDA000002000480040CE
S315080003A0014B1880704700BFD002002008B501F045
S315080003B087FB104B1B6898421AD30F4B1B7843B91F
S315080003C001220D4B1A704FF480710C4800F06CFD39
S315080003D007E00022084B1A704FF48071074800F0B6
S315080003E065FD01F06DFB064B1B881844014B186030
S315080003F008BD00BFCC020020D20200200014024033
S31508000400D002002008B54FF48071024800F04EFD76
S3150800041008BD00BF0014024038B50146074800F081
S31508000420FBFD064D01242146284600F005FE00285E
S31508000430F9D0024800F0ECFDC0B238BD003C0040DF
S3150800044070B501F03DFB00F5FA76FF252846FFF763
S31508000450E3FF0446FF2803D001F032FB8642F5D8B5
S31508000460FF2C14BF0020012070BD00BF08B5042171
S31508000470034800F019FDFF20FFF7CEFF08BD00BFB7
S31508000480000C024010B50421074800F00FFDFF20BC
S31508000490FFF7C2FFFFF7D4FF18B90446FFF7E6FFD8
S315080004A000E00124204610BD000C024038B5044681
S315080004B00D4610F0800F07D000213720FFF7F6FF12
S315080004C001283AD804F07F04FFF7D0FFFFF7DAFFD8
S315080004D048B344F04000FFF79FFF280EFFF79CFF44
S315080004E0C5F30740FFF798FFC5F30720FFF794FF0A
S315080004F0E8B2FFF791FFE4B1082C16D00120FFF708
S315080005008BFF0C2C02D1FF20FFF786FF0A24FF255C
S315080005102846FFF781FF10F0800F0ED0631E13F0F8
S31508000520FF04F5D138BDFF2038BD8720FFF774FFDB
S31508000530ECE79520FFF770FFE8E738BD38B50546C4
S315080005400C46FFF77DFF034618B32046FFF764FF06
S31508000550FD2C1DD0AC1C05F2022514F8020CFFF781
S315080005605BFF14F8010CFFF757FF0234AC42F4D1D5
S31508000570FF20FFF751FFFF20FFF74EFFFF20FFF791
S315080005804BFF00F01F00052814BF0023012300E0DD
S315080005900123184638BD00BFF8B504460D4601F0DC
S315080005A08FFA00F16407FF263046FFF735FFFF286C
S315080005B005D101F085FA8742F6D80020F8BDFE2855
S315080005C016D10234FF263046FFF726FF04F8020C40
S315080005D03046FFF721FF04F8010C0234023DF2D140
S315080005E0FF20FFF719FFFF20FFF716FF0120F8BDD0
S315080005F00020F8BD002840F06B81BB4B1B7813F038
S31508000600020F03D0B84B1878C0B270472DE9F047EF
S315080006108AB00121082000F0B1FC0121042000F075
S31508000620ADFC01214FF4004000F0B6FC4FF0040980
S31508000630CDF8009002268DF8056001278DF8047024
S3150800064000248DF807408DF80640DFF8A482694635
S31508000650404600F0DBFB4946404600F025FCA34D2A
S3150800066006220A21284600F023FC06220B212846EA
S3150800067000F01EFC06220C21284600F019FC4FF457
S31508000680E05300938DF804608DF805608DF80640F8
S315080006908DF807606946284600F0B8FBADF81040AB
S315080006A04FF48273ADF81230ADF81440ADF8164029
S315080006B0ADF818404FF40073ADF81A303023ADF892
S315080006C01C30ADF81E400723ADF82030DFF828A20D
S315080006D004A9504600F06EFC2146504600F09EFCE8
S315080006E03946504600F086FC4946404600F0DCFB99
S315080006F08DF80D608DF80C708DF80F408DF80E4052
S315080007004FF480540AA941F8204D284600F07EFB94
S315080007102146284600F0C8FB0A275446314620469B
S3150800072000F08AFC0028F9D0FF21204600F074FC6E
S3150800073001252946204600F07FFC0028F9D0013F14
S31508000740ECD14FF48053029302238DF80C308DF8C8
S315080007500D3000248DF80E408DF80F3002A963483D
S3150800076000F054FB0421624800F0A0FB2146204615
S31508000770FFF79CFE012840F0AD8001F0A1F900F5D5
S315080007807A744FF4D5710820FFF790FE012842D1FC
S3150800079009AE0AAF35464FF0FF084046FFF73CFE64
S315080007A005F8010BBD42F8D19DF82630012B40F023
S315080007B091809DF82730AA2B40F08C804FF0804816
S315080007C0A92501F07DF9844205D941462846FFF757
S315080007D06DFE0028F5D101F073F984427AD900211B
S315080007E03A20FFF763FE002874D1FF242046FFF75E
S315080007F013FE06F8010BBE42F8D19DF8243003F02B
S315080008004003DBB2002B14BF0C220422394B1A60BA
S31508000810FFF72CFE24E00021A920FFF747FE012858
S3150800082087BF01273D460227A925002601F048F97A
S31508000830844205D931462846FFF738FE0028F5D107
S3150800084001F03EF9844245D94FF400711020FFF7B4
S315080008502DFE00283ED1274B1F60FFF707FE77B312
S31508000860214A137803F0FE031370234D002128460E
S3150800087000F0C0FB0024ADF810404FF48273ADF8C9
S315080008801230ADF81440ADF81640ADF818404FF4E4
S315080008900073ADF81A30ADF81C40ADF81E400723BA
S315080008A0ADF8203004A9284600F084FB21462846E6
S315080008B000F0B4FB0121284600F09CFB04E00A4A3C
S315080008C0137843F001031370074B1878C0B207E09A
S315080008D0012070470022074B1A60FFF7C7FDEEE7B5
S315080008E00AB0BDE8F08700BF0000002000080240FB
S315080008F0000C0240D4020020003C004018B9034B0B
S315080009001878C0B270470120704700BF0000002069
S31508000910002838D170B50D461C46B3B31D4B1B785D
S3150800092013F0010F33D11C4B1B6813F0080F08BFD7
S315080009305202012C0DD111461120FFF7B7FDE0B97F
S315080009404FF400712846FFF727FEB0FA80F46409D1
S3150800095013E011461220FFF7A9FD70B94FF400768F
S3150800096031462846FFF718FE18B105F50075013C13
S31508000970F6D100210C20FFF799FDFFF777FD201C23
S3150800098018BF012070BD04207047042070BD0320E5
S3150800099070BD00BF00000020D4020020002847D107
S315080009A070B50D4616461C46002B43D0244B1B78C3
S315080009B013F0010F40D1224B1B7813F0040F3DD1E1
S315080009C0204B1B6813F0080F08BF5602012C0CD1E8
S315080009D031461820FFF76AFD20BBFE212846FFF79F
S315080009E0ADFDB0FA80F464091CE013F0060F03D0DD
S315080009F021469720FFF75AFD31461920FFF756FD85
S31508000A0080B9FC2631462846FFF798FD18B105F54A
S31508000A100075013CF6D1FD210020FFF78FFD002867
S31508000A2008BF0124FFF722FD201C18BF012070BD56
S31508000A3004207047042070BD032070BD022070BDDD
S31508000A4000000020D4020020002840F02681964BA2
S31508000A501B7813F0010F40F0228170B584B014465C
S31508000A600E2900F2FF80DFE811F00F001500FD00E7
S31508000A705C00FD00FD00FD00FD00FD00FD00B70067
S31508000A80BC00CA00D700E800FFF7FCFCB0FA80F407
S31508000A906409FEE000210920FFF708FD002840F060
S31508000AA0E38010216846FFF777FD002800F0DE8016
S31508000AB09DF800309B09012B10D19DF808209DF860
S31508000AC0093003EB02229DF807301B0403F47C135C
S31508000AD0013313449B0223600024DAE09DF80820C2
S31508000AE09DF807309B0003EB92129DF806309B0297
S31508000AF003F44063134401339DF8052002F00F0206
S31508000B009DF80A1002EBD112911C9DF8092052009B
S31508000B1002F006020A44D2B2093A9340236000243E
S31508000B20B7E0624B1B6813F0040F21D000218D201B
S31508000B30FFF7BCFC002840F09B80FF20FFF76CFC09
S31508000B4010216846FFF728FD002800F0938030251D
S31508000B50FF263046FFF760FC6B1E13F0FF05F8D141
S31508000B609DF80A301A09102393402360002490E068
S31508000B7000210920FFF79AFC00287DD1102168463C
S31508000B80FFF70AFD002879D0484B1B6813F0020FBF
S31508000B9011D09DF80A305B0003F07E039DF80B2008
S31508000BA003EBD21301339DF80D209209013A9340C5
S31508000BB0236000246DE09DF80B10CB0003F01803AA
S31508000BC003EB51119DF80A20C2F38402531C01FB62
S31508000BD00333236000245CE0344B1B681370002445
S31508000BE057E000210920FFF761FC002848D11021B1
S31508000BF02046FFF7D1FCB0FA80F4640949E00021E9
S31508000C000A20FFF753FCE8BB10212046FFF7C4FC77
S31508000C10B0FA80F464093CE000213A20FFF746FC6C
S31508000C2090BB651E0334FF263046FFF7F5FB05F833
S31508000C30010FAC42F8D100242BE01C4B1B6813F0C3
S31508000C40040F23D000218D20FFF730FC00BBFF20C6
S31508000C50FFF7E2FB40212046FFF79EFCB0FA80F43E
S31508000C60640916E0042414E0012412E0012410E0CB
S31508000C7001240EE001240CE001240AE0012408E026
S31508000C80012406E0012404E0012402E0012400E036
S31508000C900124FFF7EBFB204603E0042070470320FE
S31508000CA0704704B070BD00BF00000020D4020020C9
S31508000CB0054B1B69002B05DA034B044A5A6002F1FF
S31508000CC088325A60704700BF003C024023016745DE
S31508000CD0024A136943F0004313617047003C02401F
S31508000CE0014BD860704700BF003C02400E4BDB68E2
S31508000CF013F4803F12D10C4BDB6813F0100F0FD1A1
S31508000D00094BDB6813F0EF0F0CD1074BDB6803F0D8
S31508000D100203002B14BF07200820704701207047E4
S31508000D200520704706207047003C024000B583B096
S31508000D3008238DF80730FFF7D9FF8DF807009DF8CF
S31508000D400730DBB2012B08D1FFF7D0FF8DF807007B
S31508000D509DF80730DBB2012BF6D09DF8070003B0EB
S31508000D605DF804FB70B5054641B1012908D0022992
S31508000D700CBF4FF400764FF4407603E0002601E0FE
S31508000D804FF48076FFF7D2FF08281ED10F4C23694F
S31508000D9023F44073236123691E432661236923F0E4
S31508000DA0F8032361236943F002031D432561236980
S31508000DB043F480332361FFF7B9FF236923F0020365
S31508000DC02361236923F0F803236170BD003C0240C8
S31508000DD070B505460E46FFF7A9FF082813D10A4C39
S31508000DE0236923F440732361236943F40073236161
S31508000DF0236943F0010323612E60FFF797FF2369F8
S31508000E0023F00103236170BD003C0240F0B50023C6
S31508000E100125032605FA03F20C68A24339D10268B4
S31508000E205C0006FA04F7FF433A400260026891F84C
S31508000E3004E00EFA04FE4EEA020202600A79013A5A
S31508000E40D2B2012A17D882681740876087684A791C
S31508000E50A2403A43826047689AB205FA02FE27EA38
S31508000E600E074760D0F804E08F7907FA02F292B2CB
S31508000E7042EA0E024260C7689AB2520006FA02F2C5
S31508000E8027EA0202C260C268CF7907FA04F414435B
S31508000E90C4600133102BBDD1F0BD00BF03691942F0
S31508000EA014BF0120002070470183704741837047B3
S31508000EB010B401F007039B00C90800EB8100046A1F
S31508000EC00F21994024EA01010162016A9A400A4306
S31508000ED0026210BC704700BF10B4244B9B6803F035
S31508000EE00C03042B05D0082B06D00BBB204B036044
S31508000EF020E0204B03601DE01C4B5A685B6803F03A
S31508000F003F0312F4800F194A5268C2F3881214BFBD
S31508000F1018491749B1FBF3F303FB02F2134B5B685D
S31508000F20C3F3014301335B00B2FBF3F3036001E053
S31508000F300F4B03600D4CA368C3F303130E49CB5C38
S31508000F40DAB20368D3404360A268C2F382228A5C9D
S31508000F50D2B223FA02F28260A268C2F342328A5CF3
S31508000F60D2B2D340C36010BC704700BF00380240FD
S31508000F700024F40040787D010400002021B1054BCF
S31508000F801A6B104318637047024A136B23EA000072
S31508000F90106370470038024021B1054B1A6C1043A4
S31508000FA018647047024A136C23EA000010647047FD
S31508000FB00038024010B4038803F441540A884B8869
S31508000FC013438A881343CA8813430A8913434A89F1
S31508000FD013438A891343CA89134323439BB2038065
S31508000FE0838B23F400631B041B0C83830B8A038205
S31508000FF010BC704729B103889BB243F040030380B5
S315080010007047038823F040031B041B0C03807047BA
S31508001010808980B2704700BF8181704729B10388F3
S315080010209BB243F4005303807047038823F40053AC
S315080010301B041B0C038070470389194214BF012047
S315080010400020704730B585B004460D46038A9BB22A
S3150800105023F44053CA881343038283899BB223F43B
S31508001060B05323F00C0289882B890B4369890B43FB
S315080010709BB213438381838A9BB223F44073AA8964
S31508001080134383826846FFF727FF1C4B9C4203D015
S3150800109003F580639C4201D1039B00E0029BA28971
S315080010A012F4004F03EB830303EB8303296814BF91
S315080010B049008900B3FBF1F1114BA3FB0123580941
S315080010C00501642300FB1313A28912F4004F09D00B
S315080010D0D90032310A4AA2FB0131C1F3421242EA6F
S315080010E0050307E01B013233054AA2FB0323C3F3BA
S315080010F043132B439BB2238105B030BD001001403A
S315080011001F85EB5129B183899BB243F40053838130
S315080011107047838923F400531B041B0C8381704793
S31508001120C1F30801818070478088C0F308007047C2
S315080011300388194214BF01200020704782B0314B42
S315080011401A6842F001021A60002199601A6822F0B2
S31508001150847222F480321A602B4A5A601A6822F482
S3150800116080221A60D960009101911A6842F480328F
S315080011701A601A46136803F400330193009B01337F
S315080011800093019B1BB9009BB3F5C06FF2D11D4BB1
S315080011901B6813F4003F14BF012300230193019B2E
S315080011A0012B29D1174B9A689A609A6842F4004233
S315080011B09A609A6842F4A0529A60144A5A601A6869
S315080011C042F080721A601A46136813F0007FFBD04B
S315080011D040F203720E4B1A60A3F580639A6822F0F8
S315080011E003029A609A6842F002029A601A46936865
S315080011F003F00C03082BFAD14FF00062054B9A60F6
S3150800120002B070470038024010300024193C4005EF
S31508001210003C024000ED00E080B582B001212020AC
S31508001220FFF7ACFE01210420FFF7A8FE01214FF4C9
S315080012308020FFF7B1FE01210820FFF79FFE4FF43B
S315080012408078CDF8008000268DF8066001258DF897
S31508001250075002248DF805408DF804502F4F694633
S315080012603846FFF7D3FD41463846FFF71FFE8DF88F
S3150800127004608DF807604FF40053009369462848C8
S31508001280FFF7C4FDA7F50067072208213846FFF7D0
S315080012900FFE072209213846FFF70AFE8DF8066079
S315080012A08DF807508DF80440CDF800808DF805407C
S315080012B069463846FFF7AAFD8DF804404FF40073D7
S315080012C0009369463846FFF7A1FD29462046FFF7F1
S315080012D055FEA7F50067092208213846FFF7E8FDFD
S315080012E0092211463846FFF7E3FD4FF44073009391
S315080012F08DF804408DF805408DF806608DF8075086
S3150800130069463846FFF782FD29464FF00070FFF719
S3150800131043FE00F0D9FC00F0E7FCFCE700140240AD
S3150800132000080240F8B54A4A02F1240E00264FF496
S31508001330FA7747F23050157854782B1903FB077360
S3150800134090FBF3F103FB110139B990FBF3F39EB25D
S31508001350731E9BB2B3F5806F03D302329645EAD16A
S315080013606EE03C4B00225A611A6842F400421A6049
S315080013701B6813F4004F06D0364F00F031FD3B686A
S3150800138013F4004FF9D1334B1A6822F002021A609F
S315080013901A6842F001021A605B6813F0010F06D161
S315080013A02C4F00F01DFD7B6813F0010FF9D0013DAD
S315080013B0013C240544EA0545731E1D43254AD561AB
S315080013C0136823F001031360536813F0010F06D066
S315080013D0144600F005FD636813F0010FF9D11D4BA3
S315080013E0D3F8002242F00102C3F80022D3F81C22E7
S315080013F022F00102C3F81C22D3F80C2242F00102A3
S31508001400C3F80C220022C3F84022C3F84422D3F8BA
S31508001410042222F00102C3F80422D3F8142222F08F
S315080014200102C3F81422D3F81C2242F00102C3F8C1
S315080014301C22D3F8002222F00102C3F80022F8BDCC
S31508001440EC21054800F00AFC00252C4689E700BF78
S31508001450A0490008006400407849000838B50446E9
S315080014600D46224B9B6813F0806F04D14FF4A07190
S315080014701F4800F0F3FB1D4BD3F8802102F0010250
S31508001480C3F88021D3F8802142F07C4242F400124E
S31508001490C3F88021C3F88451E078A1780A0442EAA7
S315080014A0006122780A43617842EA0122C3F888215A
S315080014B0E079A1790A0442EA006122790A4361794E
S315080014C042EA0122C3F88C21D3F8802142F00102B6
S315080014D0C3F880219B6813F0806F06D1034C00F097
S315080014E07FFCA36813F0806FF9D038BD0064004014
S315080014F0784900081B4BDB6813F0030F2FD0194BF4
S31508001500D3F8B02140F26763B3EB525F20D1154B95
S31508001510D3F8B8210270D3F8B821120A4270D3F86A
S31508001520B821120C8270D3F8B821120EC270D3F803
S31508001530BC210271D3F8BC21120A4271D3F8BC212E
S31508001540120C8271D3F8BC311B0EC371012000E066
S315080015500020044AD36843F02003D3607047002074
S31508001560704700BF0064004008B500F0DBF908BD0D
S3150800157010B500F06DFAA0B1FEF76CFE88B100F068
S31508001580EBFB00F089FA00F067FA20F0604020F0E3
S315080015907F00044B186000F05FFA446800F0C4F955
S315080015A0A04710BD08ED00E072B170B50D46561E95
S315080015B0B6B2441E064415F8013B04F8013F00F094
S315080015C00FFCB442F7D170BD704700BF70B5064630
S315080015D00B4D002400F004FC2B68B3420AD86A6855
S315080015E013449E4206D204EB4401054B03EB8101EA
S315080015F0087A70BD01340C35062CEBD1FF2070BD7E
S31508001600DC4900082DE9F84380460068FFF7DEFF4D
S31508001610FF282FD0FFF74CFBF320FFF761FBFFF7FE
S3150800162065FB012818BF002404D1FFF751FB0020F1
S31508001630BDE8F883D8F8007004EB0709251D58F8AB
S31508001640056000F0CDFB31464846FFF7C1FB082888
S3150800165008D1E3599E4207D12C46B5F5007FE9D15A
S31508001660012402E0002400E00024FFF731FB2046B5
S31508001670BDE8F8830020BDE8F88300BF38B50D46FD
S31508001680114B984207D00446104B994208D0FFF7F1
S31508001690B9FF08B911E00E4CC5F308037BB900E0A1
S315080016A0094C2368AB420CD0204640F8045B4FF443
S315080016B000722946FFF778FF03E0002038BD0020B6
S315080016C038BD204638BD00BFD8020020008000087B
S315080016D0DC0400202DE9F04106460C4617461D4657
S315080016E021F4FF7828F001080368B3F1FF3F06D11B
S315080016F040F8048B4FF400724146FFF755FF3368F4
S31508001700984505D041463046FFF7B8FF0646E0B192
S315080017103368E41A3444043408F5007800F060FBB2
S31508001720331DE31AB3F5007F06D341463046FFF76B
S31508001730A5FF064660B1041D17F8013B04F8013BF6
S31508001740013DEBD10120BDE8F0810020BDE8F08124
S315080017500020BDE8F08100BF4FF0FF33024A136056
S31508001760024A1360704700BFDC040020D80200203C
S3150800177070B504460D461646FFF728FFFF2814D015
S31508001780681E2044FFF722FFFF2810D024F4FF73B9
S3150800179023F00103074A93422B46324621460CBFE3
S315080017A005480648FFF796FF70BD002070BD00206B
S315080017B070BD00BF00800008D8020020DC040020AD
S315080017C0F8B506460D46FFF701FF0446681E304485
S315080017D0FFF7FCFE84422AD80546A31EDBB2FC2B83
S315080017E027D8072827D8FFF763FAF320FFF778FAF0
S315080017F0FFF77CFA012803D1FFF76AFA0020F8BD43
S315080018000E4F022600F0ECFA314637F81400FFF7BF
S31508001810A9FA082803D0FFF75BFA0020F8BD0134BF
S31508001820E4B2A542EED2FFF753FA0120F8BD002034
S31508001830F8BD0020F8BD0020F8BD00BFC449000867
S31508001840114B1B68B3F1FF3F18D000B583B00E4BA0
S3150800185059689A681144DA6811441A6911445A6930
S3150800186011449A691144DA698B185B4202AA42F854
S31508001870043D04210548FFF77BFF01E0012070477E
S3150800188003B05DF804FB00BFD8020020848100087D
S315080018900D4B1A6804331B6813440C4A1268134428
S315080018A00B4A126813440B4A11680B440432126837
S315080018B01A44094B1B681344084A1268D3420CBFE2
S315080018C001200020704700BF00800008088000083B
S315080018D00C80000810800008188000088481000821
S315080018E008B50C4B1B68B3F1FF3F04D00948FFF756
S315080018F089FE034660B1084B1B68B3F1FF3F06D06B
S315080019000548FFF77FFE031C18BF012300E00123EB
S31508001910184608BDD8020020DC040020004870479D
S315080019200080000872B6704762B6704707498D4650
S315080019300749084A084B9A42BEBF51F8040B42F8B9
S31508001940040BF8E705488047054800470080002053
S315080019508851000800000020840000203D1100087E
S31508001960E10100083249334A002301E041F8043B0B
S315080019709142FBD3FFF750FCFEE7FEE7FEE7FEE7E2
S31508001980FEE7FEE7FEE7FEE7FEE7FEE7FEE7FEE721
S31508001990FEE7FEE7FEE7FEE7FEE7FEE7FEE7FEE711
S315080019A0FEE7FEE7FEE7FEE7FEE7FEE7FEE7FEE701
S315080019B0FEE7FEE7FEE7FEE7FEE7FEE7FEE7FEE7F1
S315080019C0FEE7FEE7FEE7FEE7FEE7FEE7FEE7FEE7E1
S315080019D0FEE7FEE7FEE7FEE7FEE7FEE7FEE7FEE7D1
S315080019E0FEE7FEE7FEE7FEE7FEE7FEE7FEE7FEE7C1
S315080019F0FEE7FEE7FEE7FEE7FEE7FEE7FEE7FEE7B1
S31508001A00FEE7FEE7FEE7FEE7FEE7FEE7FEE7FEE7A0
S31508001A10FEE7FEE7FEE7FEE7FEE7FEE7FEE7FEE790
S31508001A20FEE7FEE7FEE7FEE7FEE7FEE7FEE7FEE780
S31508001A3084000020EC0F002008B5FFF78DFE08BDD6
S31508001A4008B5FFF795FE08BD08B5FFF7B9FE08BD4E
S31508001A5008B5FFF71DFF08BD08B5FFF75FFF08BD0E
S31508001A6008B5FFF7EDFE034610B1FFF739FF034649
S31508001A70184608BD054B00221A60054959609A6048
S31508001A8005211960034B1A60704700BF10E000E09B
S31508001A90BFD40100E00600200022014B1A607047FF
S31508001AA010E000E0044B1B6813F4803F03D0034AA0
S31508001AB0136801331360704710E000E0E006002069
S31508001AC008B5FFF7EFFF014B186808BDE0060020D0
S31508001AD038B5044680210A48FFF72AFB68B1214633
S31508001AE00748FFF71DFB064D802421462846FFF7C9
S31508001AF01FFB0028F9D0012038BD002038BD00BFE3
S31508001B000048004010B5044620210648FFF710FBA0
S31508001B10012805D10348FFF707FB2070012010BDF7
S31508001B20002010BD0048004010B584B04FF4614352
S31508001B3000930023ADF80430ADF80630ADF8083050
S31508001B40ADF80C300C23ADF80A30054C6946204632
S31508001B50FFF778FA01212046FFF7D4FA04B010BD42
S31508001B6000480040F8B505460C46402903D97521BA
S31508001B70114800F073F82046FFF7AAFF012803D0A2
S31508001B8079210D4800F06AF8A3B29BB16C1E013B9F
S31508001B909BB21D44084F822600F022F914F8010F63
S31508001BA0FFF796FF012803D03146384600F056F86D
S31508001BB0AC42F1D1F8BD00BF244A000838B5224B23
S31508001BC01C789CB92148FFF79DFF012839D11F4B86
S31508001BD01B78002B30D0FFF773FF1D4B18600022CF
S31508001BE01C4B1A700122184B1A702AE00546194B2D
S31508001BF01878194B1844FFF785FF0446012810D1B9
S31508001C00144B1A780132D2B21A70104B1B789342D1
S31508001C1014D111492846FFF7C7FC00220A4B1A704F
S31508001C200FE0FFF74DFF0A4B1B686433984207D94C
S31508001C300024054B1C7004E01C4602E0002400E06A
S31508001C400024204638BD00BF2A070020E8060020E9
S31508001C50E406002029070020E906002008B500F060
S31508001C60BFF8FCE708B500F0B3F8012816D000F075
S31508001C7041F998B10A4B1B78012B0FD1FFF720FFCA
S31508001C80084B1B6803F5FA73984207D30022044BE6
S31508001C901A7000F037F908B9FFF76AFC08BD00BFEB
S31508001CA02B0700202C07002008B50122044B1A70C8
S31508001CB0FFF706FF034B1860FFF7D4FF08BD00BF08
S31508001CC02B0700202C07002008B5FFF74DFC00F075
S31508001CD083F8FFF7CFFEFFF7AFFE00F0F5F800F048
S31508001CE00FF8FFF7E1FF08BD08B500F079F8FFF730
S31508001CF0D9FE00F025FA00F013F8FFF7B3FF08BD88
S31508001D0010B502F025FCFFF70DFB044C01232370E8
S31508001D10FFF70AFF0023237010BD00BF1400002040
S31508001D2008B50B48FFF7E6FB012805D10122094B48
S31508001D301A70074802F02AFC0548FFF73FFF0128FA
S31508001D4005D10022034B1A70014802F01FFC08BD9A
S31508001D503007002014000020704700BF38B504463D
S31508001D600D46084B1B78012B02D1C9B2FFF776FB4B
S31508001D70044B1B781BB9E9B22046FFF7F3FE02F0C5
S31508001D80FDFB38BD14000020074B1B78022B06D03C
S31508001D90032B06D0012B0CBF0820402070470020DB
S31508001DA070470020704700BF14000020074B1B78BF
S31508001DB0022B06D0032B06D0012B0CBF082040208F
S31508001DC07047002070470020704700BF14000020AD
S31508001DD008B502F0CBFB08BD08B5FEF749FA08BD01
S31508001DE008B5FEF74BFA08BD00F00F03092802D91B
S31508001DF003F13700704703F13000054B1B680344B5
S31508001E005B7803F00303022B08BF2038C0B2704783
S31508001E101800002038B505460C460009FFF7E4FF10
S31508001E20207005F00F00FFF7DFFF60700023A37036
S31508001E30204638BD10B4034602460C480131A0FBC3
S31508001E400242D208FAD100220A70084CA4FB030207
S31508001E50D20802EB8200A3EB4003303301F8013DC0
S31508001E601346002AF2D1084610BC7047CDCCCCCC1C
S31508001E7070B4144B1E68441E451C002014F8013F1C
S31508001E80F218517801F00301022908BF203BDBB2A2
S31508001E90A3F13002D2B2162A0FD8A3F13A01C9B279
S31508001EA006290CD9092A84BF373BDAB202EB00139C
S31508001EB003F0FF00AC42E1D102E0002000E0002080
S31508001EC070BC70471800002008B50022054B1A7030
S31508001ED00549064801F022FE18B177210448FFF7A4
S31508001EE0BDFE08BDB0070020504A0008BC07002008
S31508001EF0544A0008024B1878B0FA80F04009704737
S31508001F00B007002008B5FFF763FF01280AD0084B81
S31508001F101B784BB9FEF7B6F9012807D10122044B05
S31508001F201A7008BD002008BD002008BD002008BDA5
S31508001F30B00700200378114A1168CA18527802F0CF
S31508001F400302022A08BF203B532B0ED143781944BB
S31508001F504A7812F0040F0AD0312B0AD0322B0AD055
S31508001F60332B0CBF02200320704703207047032041
S31508001F707047002070470120704700BF18000020F6
S31508001F8070B506460230FFF773FF054684B204367D
S31508001F903046FFF76DFF2844C5B2013CA4B20236AD
S31508001FA0012CF5D83046FFF763FFED43EDB28542C5
S31508001FB014BF0020012070BD2DE9F04104461646E5
S31508001FC0884601B120B940F261215C48FFF746FE18
S31508001FD02046FFF7AFFF0546032800F0928020460B
S31508001FE0FFF7CEFF002800F08F80012D28D015B10D
S31508001FF0022D52D08CE0A01CFFF73AFF0746201DA1
S31508002000FFF736FF0502C8F80050A01DFFF730FF9E
S315080020102844C8F800000834F81E07B2002E7AD003
S31508002020B846002F7ADD00252046FFF721FF7055B8
S3150800203002340135ADB24545F6DB3846BDE8F081D8
S31508002040A01CFFF715FF0746201DFFF711FF050423
S31508002050C8F80050A01DFFF70BFF05EB0025C8F8D0
S31508002060005004F10800FFF703FF2844C8F80000F1
S315080020700A34381F07B2002E53D0B846002F53DD56
S3150800208000252046FFF7F4FE705502340135ADB23F
S315080020904545F6DB3846BDE8F081A01CFFF7E8FEAB
S315080020A00746201DFFF7E4FE0506C8F80050A01DE8
S315080020B0FFF7DEFE05EB0045C8F8005004F10800FE
S315080020C0FFF7D6FE05EB0025C8F8005004F10A0014
S315080020D0FFF7CEFE2844C8F800000C34781F07B274
S315080020E02EB3B846002F25DD00252046FFF7C0FE93
S315080020F0705502340135ADB24545F6DB3846BDE8C4
S31508002100F0810020BDE8F0814FF0FF30BDE8F08196
S315080021100020BDE8F0813846BDE8F0813846BDE8C4
S31508002120F0813846BDE8F0813846BDE8F08138468A
S31508002130BDE8F0813846BDE8F08100BF544A000882
S31508002140F8B5AF4B1B78002B00F0EC81012B29D199
S31508002150FFF772FCFEF7B8F8AA48FEF7F9F8AA489E
S31508002160FEF7F6F8FEF7ACF801220146A74801F09B
S3150800217007FD30B1A648FEF7EBF80120FEF7DCF8BC
S31508002180F8BDA448FEF7E4F8A348FEF7E1F8A3482B
S31508002190FEF7DEF8A24B00221A605A600222984B1C
S315080021A01A70F8BD022B40F0F5809E4C04F50C72AF
S315080021B04FF480719C4802F0FBF894F841326BB1F9
S315080021C09348FEF7C5F80220FEF7B6F804F50C703A
S315080021D001F0A2FF00228A4B1A70F8BD002877D0BA
S315080021E09148002200F5C071FFF7E6FE0446B0F1FB
S315080021F0FF3F0CD18648FEF7ABF80320FEF79CF8A4
S31508002200824801F089FF00227D4B1A70F8BD00282C
S315080022105EDD834B5B6833B9814B834AD2F88021F4
S315080022201A60586054E07E4A12681A447E49D1F80A
S315080022308011914203D10344794A536048E07548B6
S31508002240FEF786F87948FEF783F8794D744E2946E5
S315080022507068FFF7EFFD2846FEF77AF87548FEF72F
S3150800226077F837682946380EFFF7D4FDA91CC7F357
S315080022700740FFF7CFFD291DC7F30720FFF7CAFD63
S31508002280A91DF8B2FFF7C6FD2846FEF761F86A48A9
S31508002290FEF75EF871683068FFF7D6FB60B95C48F0
S315080022A0FEF756F80520FEF747F8584801F034FFC0
S315080022B00022534B1A70F8BD5648FEF749F857489E
S315080022C0FEF746F8564B584AD2F880211A605C60E9
S315080022D0544BD3F84422D3F83C329A4240F0228138
S315080022E000214A4801F02AFF60B14948FEF730F854
S315080022F00420FEF721F8454801F00EFF0022404B66
S315080023001A70F8BD464B5B68002B3CD04148FEF777
S315080023101FF84648FEF71CF8454C414D21466868AB
S31508002320FFF788FD2046FEF713F84248FEF710F837
S315080023302E682146300EFFF76DFDA11CC6F3074037
S31508002340FFF768FD211DC6F30720FFF763FDA11DF2
S31508002350F0B2FFF75FFD2046FDF7FAFF3648FDF7B6
S31508002360F7FF69682868FFF76FFB60B92848FDF72B
S31508002370EFFF0520FDF7E0FF244801F0CDFE00221F
S315080023801F4B1A70F8BD2348FDF7E2FF03221C4BCA
S315080023901A70F8BD032B40F0C580224C04F50C7268
S315080023A04FF48071204802F003F894F841326BB17B
S315080023B02248FDF7CDFF0220FDF7BEFF04F50C709D
S315080023C001F0AAFE00220E4B1A70F8BD00287CD038
S315080023D0154800F5807200F5C071FFF7EDFD064659
S315080023E0B0F1FF3F2ED11648FDF7B2FF0320FDF7E7
S315080023F0A3FF064801F090FE0022014B1A70F8BDB3
S31508002400B0070020704A0008944A0008EC0900202A
S31508002410BC4A0008C44A0008CC4A0008F04A00082A
S31508002420B4070020BC070020140C0020204B00082D
S31508002430700700202C4B0008D04B0008484B0008BA
S315080024406C4B0008002840DD3748FDF781FF374C04
S3150800245021463046FFF7EEFC2046FDF779FF344863
S31508002460FDF776FF334D214695F88301FFF7D2FC39
S31508002470A11C95F88201FFF7CDFC211D95F8810175
S31508002480FFF7C8FCA11D95F88001FFF7C3FC20469D
S31508002490FDF75EFF2848FDF75BFF05F580723146BC
S315080024A0D5F88001FFF7CCFA60B92448FDF750FF4C
S315080024B00620FDF741FF224801F02EFE0022214B9F
S315080024C01A70F8BD2048FDF743FF204BD3F8442285
S315080024D0D3F83C329A4225D11D48FDF739FFFFF75C
S315080024E0BFFA60B91548FDF733FF0720FDF724FF4B
S315080024F0134801F011FE0022124B1A70F8BD12485B
S31508002500FDF726FF1348FDF723FF0D4801F004FEEB
S315080025101148FDF71DFF00220A4B1A70FDF7E8FE69
S31508002520FFF726F8F8BD00BF904B0008700700209B
S31508002530A04B0008140C0020D04B0008BC4A000829
S31508002540EC090020B0070020C44A0008BC07002098
S31508002550B84B0008D44B0008EC4B0008C2788378C7
S3150800256043EA0222437843EA0223007840EA03203A
S31508002570704700BF3AB101388A1811F8013B00F8D4
S31508002580013F9142F9D1704702394369023B9942AA
S315080025903DBF4389806A01FB03000020704700BFE6
S315080025A000F10B010023DA0142EA530310F8012B6C
S315080025B0134403F0FF038842F5D11846704700BF5D
S315080025C00168E1B110B40C781F2C09D93A2C1FD038
S315080025D00A4612F8013F1F2B04D93A2BF9D105E018
S315080025E023460A463A2B18BF002013D14B1C9A42A1
S315080025F008D1302C09D10231016000200AE04FF0E1
S31508002600FF3070474FF0FF3004E04FF0FF3001E035
S315080026100A46EBE710BC704738B50C4670B105465C
S3150800262003685BB11A784AB1D9888288914205D184
S315080026305878FEF763F910F0010F03D000232360E2
S31508002640092038BD2B682360002038BDC37833B312
S315080026502DE9F0410446C56A00F1300701232A46F0
S3150800266039464078FEF79AF9D8B90023E370236A09
S31508002670EB1AA269934217D2A678012E17D94FF002
S315080026800108A3691D4443462A4639466078FEF781
S3150800269085F9013E012EF4D10020BDE8F081002025
S315080026A070470120BDE8F0810020BDE8F0810020D8
S315080026B0BDE8F08170B5C36A8B4213D004460D4657
S315080026C0FFF7C4FF064670B901232A4604F1300114
S315080026D06078FEF71DF900281CBF01264FF0FF356C
S315080026E0E56200E00026304670BD00BF10B504461E
S315080026F0FFF7ACFF0346002852D12378032B47D1B6
S315080027002379012B44D104F1300104F50C700B46F2
S31508002710002203F8012B8342FBD1552384F82E327D
S31508002720AA2384F82F32522384F8303084F83130C3
S31508002730612384F83230412284F83320722084F8E9
S31508002740140284F8150284F8162284F817322369CD
S3150800275084F818321A0A84F819221A0C84F81A22EC
S315080027601B0E84F81B32E36884F81C321A0A84F8B4
S315080027701D221A0C84F81E221B0E84F81F32E269E9
S315080027800132E26201236078FEF708F9002323711B
S31508002790002211466078FEF757F9031C18BF01237B
S315080027A0184610BD2DE9F843012940F28380436994
S315080027B0994280F0818017460C4605460378022B1D
S315080027C03DD0032B51D0012B78D101EB5108016A7A
S315080027D001EB5821FFF76EFF0646002840F085807A
S315080027E008F10109C8F3080814F0010F13D0A8442A
S315080027F098F8303003F00F0343EA071388F83030AF
S315080028000123EB70296A01EB59212846FFF752FF8D
S31508002810002859D054E0A84488F830700123EB709A
S31508002820296A01EB59212846FFF744FF002850D0B2
S3150800283048E0A94489F830200123EB7055E0016A85
S3150800284001EB1421FFF736FF064600284DD1630039
S3150800285003F4FF73EA1882F830701346C7F30722A9
S3150800286083F831200123EB703FE0016A01EBD411B4
S31508002870FFF720FF0646C0BB27F07047A40004F404
S31508002880FE7404F13008A8444046FFF767FE00F0DE
S31508002890704040EA07022C4484F83020130A88F86E
S315080028A00130130C88F80230120E88F80320012331
S315080028B0EB701AE0022618E0022616E0022614E05B
S315080028C0064612E0064610E0C9F30809C7F30712E0
S315080028D0AFE7C9F3080905EB090393F8303023F08D
S315080028E00F03C7F303221A43A3E73046BDE8F8836C
S315080028F08A76C2F30723CB760378032B03D1120C0F
S315080029000A75120A4A7570472DE9F84300238B7534
S315080029108369002B72D00D460646436AB3F1FF3F22
S315080029201DD0836A9F1C188888B101F115080024F8
S31508002930A146494601F092FD58B1FF2C0BD001344F
S3150800294008F8010F37F8020B0028F2D104E000243A
S3150800295002E0002400E000242C440023A375A87D8F
S31508002960002423462E275A1CF169CB5C202B22D043
S31508002970052B08BFE523092A05D108B929198F753A
S3150800298029194F72013429194B7298B9A3F14101DB
S31508002990C9B219290CD8F169097B082A8CBF4FF0EE
S315080029A0100E4FF0080E1EEA010F1CBF2033DBB2D3
S315080029B029198B75013413460B2AD4D138B92B192A
S315080029C000229A75F3691B7B934208BF14462C4470
S315080029D000236372F369DB7A2B72F0691C30FFF708
S315080029E0BDFD2860F269517E137E43EA0123AB8060
S315080029F0F269D17D937D43EA0123EB80BDE8F88334
S31508002A00012955D9F8B506687369994252D20C4618
S31508002A103378022B29D0032B39D0012B4CD101EB6B
S31508002A205105316A01EB55213046FFF743FE002870
S31508002A3044D16F1CC5F30805354495F83050316A02
S31508002A4001EB57213046FFF735FE002839D1C7F389
S31508002A5008073E4496F8300045EA002014F0010FB6
S31508002A6014BF0009C0F30B00F8BD316A01EB14214D
S31508002A703046FFF71FFE38BB610001F4FF7173187B
S31508002A8093F8310093F8303043EA0020F8BD316AF4
S31508002A9001EBD4113046FFF70DFEC0B9A00000F4D3
S31508002AA0FE7030303044FFF759FD20F07040F8BD15
S31508002AB0012070470120F8BD0120F8BD4FF0FF3016
S31508002AC0F8BD4FF0FF30F8BD4FF0FF30F8BD4FF0BE
S31508002AD0FF30F8BDB1F5001F46D22DE9F041064694
S31508002AE00C4611F01F0F41D1D0F80080316185687E
S31508002AF085B998F80030022B02D9D8F8243043B9A2
S31508002B00B8F80830B3EB541F33D9D8F82430B3617A
S31508002B101BE01D46B8F80A707F02BC4210D329464E
S31508002B203046FFF76DFF0546B0F1FF3F24D0012878
S31508002B3025D9D8F81430984224D2E41BA742EED9F6
S31508002B4029464046FFF720FDB0617561B369E3B1D8
S31508002B5003EB5423B36108F13003C4F30804234498
S31508002B60F3610020BDE8F081022070470220BDE82D
S31508002B70F0810220BDE8F0810120BDE8F081022045
S31508002B80BDE8F0810220BDE8F0810220BDE8F081B1
S31508002B902DE9F04107460668884631B9F56885B1DA
S31508002BA073699D4228BF01250CE0FFF729FF01281C
S31508002BB046D9B0F1FF3F46D07369984252D345468D
S31508002BC000E001252C46013473699C4202D3012D8D
S31508002BD03DD9022421463846FFF712FF38B10128AD
S31508002BE038D0B0F1FF3F38D0AC42ECD139E04FF0E5
S31508002BF0FF3221463046FFF7D5FD0346C8B9B8F17E
S31508002C00000F06D0224641463046FFF7CBFD034665
S31508002C1078B9F46033697269023A93423CBF03F1AA
S31508002C20FF333361337943F0010333712046BDE83E
S31508002C30F081012B0CBF4FF0FF300120BDE8F08179
S31508002C400120BDE8F0814FF0FF30BDE8F08100209B
S31508002C50BDE8F0810120BDE8F0814FF0FF30BDE806
S31508002C60F0810020BDE8F0812DE9F0410E460129EA
S31508002C7030D907461146046863699E422DD22AB1A7
S31508002C804FF0FF322046FFF78DFD48BB4FF0000896
S31508002C9031463846FFF7B4FE054618B3012824D056
S31508002CA0B0F1FF3F24D0424631462046FFF77AFD71
S31508002CB008BB2369B3F1FF3F05D0013323612379AC
S31508002CC043F0010323712E4663699D42E0D3002039
S31508002CD0BDE8F0810220BDE8F0810220BDE8F08160
S31508002CE0BDE8F0810020BDE8F0810220BDE8F08152
S31508002CF00120BDE8F081BDE8F08100BF8369002BA3
S31508002D0076D02DE9F04705692035B5F5001F71D253
S31508002D10884604460668C5F30807002F61D10133C3
S31508002D208361416941B93389B3EB551F59D80023EB
S31508002D3083610420BDE8F0877389013B13EA5523B4
S31508002D404FD1FFF75DFE8146012856D9B0F1FF3F06
S31508002D5056D0736998423DD3B8F1000F04D10023C9
S31508002D60A3610420BDE8F08761692046FFF710FFDC
S31508002D708146002847D0012848D0B0F1FF3F48D007
S31508002D803046FFF763FC002846D106F1300306F506
S31508002D900C71002203F8012B8B42FBD149463046C1
S31508002DA0FFF7F2FBF0624FF000084FF0010A0AE065
S31508002DB086F803A03046FFF749FC80BB08F10108F6
S31508002DC0F36A0133F36273899845F1D3F36AC8EB62
S31508002DD00303F362C4F8149049463046FFF7D4FB60
S31508002DE0A061256130373744E7610020BDE8F087E8
S31508002DF0042070470420BDE8F0870220BDE8F0876C
S31508002E000120BDE8F0870720BDE8F0870220BDE86D
S31508002E10F0870120BDE8F0870120BDE8F087012092
S31508002E20BDE8F0872DE9F843044605680669416A56
S31508002E30B1F1FF3F03D0FFF74DFE0346D8B94FF077
S31508002E40E50801274FF00009A1692846FFF732FC7B
S31508002E50034668B9E26982F80080EF7022699642F3
S31508002E6009D949462046FFF749FF03460028EBD013
S31508002E70042B08BF02231846BDE8F8832DE9F04F56
S31508002E8085B00546D0F800B00021FFF723FE0028DC
S31508002E9040F0A6804FF0FF336B624FF0FF0AD14631
S31508002EA01F46A9695846FFF705FC002840F0998097
S31508002EB0EC692678002E00F09580E37A03F03F024D
S31508002EC0AA71E52E04D013F0080F05D00F2A05D0F5
S31508002ED06F624FF0FF097BE00F2A5AD1D5F8288098
S31508002EE0B8F1000F74D016F0400F06D094F80DA074
S31508002EF006F0BF062B696B6204E0B14518BF4FF0B8
S31508002F00FF0965D1637B009353455FD1E27EA37EBB
S31508002F1053EA02237DD1237803F03F03013B03EBF9
S31508002F20430203EB8203DFF80CA10121CDF804B0BC
S31508002F3003961E4602951AF8013BE2185578E35C9B
S31508002F4043EA052581B1FE2E58D8284601F0A8FA8D
S31508002F50834606F1010938F8160001F0A1FA8345FF
S31508002F6050D129464E4603E04FF6FF739D424DD198
S31508002F702F4B5345DFD1DDF804B03246039E029D40
S31508002F80237813F0400F33D091B338F812307BB35F
S31508002F903FE0B9F1000F04D12046FFF701FB824557
S31508002FA022D02A6AD37A13F0010F37D00AE011F833
S31508002FB0013B10F8012B9B1A8C4202D0002BF6D04D
S31508002FC000E09BB16F624FF0FF0901E04FF0FF0987
S31508002FD000212846FFF792FE00283FF462AF24E05E
S31508002FE023E022E0042020E000201EE000201CE070
S31508002FF0013E5FFA86F9DDF800A0E9E7DDF804B0DE
S31508003000029D06E0DDF804B0029D02E0DDF804B09A
S31508003010029DDDF800A04FF0FF09D9E7611C501C9E
S3150800302014F80B3B12789B1AC8E705B0BDE8F08F79
S31508003030B94C0008AC4C00082DE9F04F8BB0076A74
S31508003040FB7A13F0A00F40F03E81D0F828A0BAF81A
S3150800305000304BB153464FF0000808F1010833F829
S31508003060022F002AF9D101E04FF000080446036850
S3150800307001930C22394607A8FFF77CFA9DF82730FA
S3150800308013F0010F75D00023FB72A3620B2207A968
S315080030903846FFF76FFA012633464FF07E0920259A
S315080030A01FE00B2207A93846FFF764FA052E17D941
S315080030B0AAF1020E33460EE0102102F0010000EBE1
S315080030C04303520813F4803F1CBF83F4883383F00C
S315080030D021030139F1D13EF8022F002AECD100E094
S315080030E033460DF11C0E072203F00F0000F13001E4
S315080030F0392988BF00F13701013A0EF8011D1B096D
S31508003100F2D10AAB134403F8149C62B13B78202B26
S315080031100BD03946002301339A4207D011F8010F24
S315080031202028F8D102E0002300E00023F918013333
S31508003130072A05D80AA8104410F8140C013200E032
S31508003140284601F8010B072BF1D92046FFF796FE12
S3150800315020B90136642EA4D10720D3E0642E00F0EE
S31508003160B480042840F0B3809DF82730FB72C4F879
S3150800317028A09DF8273013F0020F07D008F10C0895
S31508003180624DA5FB0835AD08013500E00125276825
S3150800319000212046FFF79EFC0346002840F0AC803D
S315080031A000264FF00108A1693846FFF783FA03465F
S315080031B0002840F0A180E3691B78E52B00D01BB9F5
S315080031C00136B54201D19AE0002641462046FFF76E
S315080031D095FD03460028E6D08EE02169A1EB45114E
S315080031E02046FFF777FC034600287CD1206AFFF7C4
S315080031F0D7F9029000260396A1690198FFF75AFAB3
S31508003200034600286FD1D4F82880E1695FFA85F96A
S315080032109DF808304B734FF00F03CB720E738E7602
S31508003220CE7609F1FF3303EB430003EB8000384AFF
S3150800323002F10D0C039B4FF6FF774FF0FF0ABB42D6
S3150800324048D000F1010E38F81030107801EB000B69
S315080032500B54180A8BF8010013B970463B4600E078
S31508003260704601326245EAD14FF6FF72934202D0A8
S3150800327038F810300BB949F0400981F8009001235D
S31508003280019AD37031462046FFF738FD034650BBF6
S31508003290013DB1D129E0E36903F12001002203F8D9
S315080032A0012B9942FBD10B22216AE069FFF762F9EB
S315080032B0E269236ADB7A03F0180313730123019A80
S315080032C0D37000201EE006201CE007201AE019E053
S315080032D0072017E092F800E001EB0E0B01F80EA0AC
S315080032E08BF801A0BDE718460CE0A1690198FFF725
S315080032F0E1F90028CFD005E0042BE9D0F3E7013D3A
S31508003300F3D06AE70BB0BDE8F08F00BF4FECC44EB0
S31508003310AC4C000810B504460023C3704FF0FF33C9
S31508003320C362FFF7C7F9F0B994F82F2294F82E3242
S3150800333043EA02231BB20F4A934216D104F16600F0
S31508003340FFF70CF920F07F400B4B98420FD004F1A1
S315080033508200FFF703F920F07F40074B984214BF1D
S315080033600220002010BD042010BD032010BD00203F
S3150800337010BD00BF55AAFFFF464154002DE9F04392
S3150800338085B00E46174600230B60FFF719F9051E90
S31508003390C0F22E81C04B53F82540002C00F02A813C
S315080033A0346007F0FE07237883B16078FDF7A6FA44
S315080033B010F0010F0AD1002F00F01E8100F0040062
S315080033C0C0B200280CBF00200A206FE1002323703A
S315080033D0E8B26070FDF70EF910F0010F40F00E81AB
S315080033E01FB110F0040F40F00B8100212046FFF7B3
S315080033F091FF022825D16E4604F5FB7504F236289E
S315080034006F464FF0000915F8043C1BB12846FFF734
S31508003410A5F800E0484647F8040B1035A845F2D150
S3150800342004AF4FF0030856F8045B35B12946204629
S31508003430FFF770FF012801D802E14046BE42F2D1EB
S3150800344000E00025042800F0DD80012888BF0D2053
S3150800345000F22C8194F83C2094F83B3043EA02238E
S315080034601BB2B3F5007F40F0CF8094F8477094F80C
S31508003470463053EA072704D104F15400FFF76EF8E3
S315080034800746A76194F8409084F8029009F1FF3343
S31508003490DBB2012B00F2BA8094F83D60B3B26381C7
S315080034A0002B00F0B580731E334240F0B38094F8C9
S315080034B0428094F8413043EA0828A4F8088018F0B6
S315080034C00F0F40F0A98094F8440094F8433053EA6B
S315080034D0002003D104F15000FFF740F894F83F208C
S315080034E094F83E3053EA022300F0988007FB09F966
S315080034F003EB181149448842C0F09280401AB0FB89
S31508003500F6F6002E00F08E8040F6F572964294BFCD
S31508003510012202224FF6F570864200F295800236A5
S315080035206661E5612B4423622944A162032A15D109
S3150800353094F85B2094F85A3053EA022374D1B8F110
S31508003540000F73D104F15C00FFF708F86062B3005E
S3150800355003F2FF13B7EB532F6AD38AE0B8F1000FD3
S3150800356068D04B446362022A0FBF760006EB460317
S3150800357006F0010606EB530675E0691C2046FFF7C0
S3150800358099F828BB0023237194F82F2294F82E3239
S3150800359043EA02231BB2414A93421BD104F130008D
S315080035A0FEF7DCFF3E4B984216D104F50570FEF790
S315080035B0D5FF3C4B984211D104F50670FEF7CEFFB5
S315080035C0206104F50770FEF7C9FFE060032206E0F4
S315080035D0032204E0032202E0032200E00322227011
S315080035E0314A138801339BB21380E38000205DE0E3
S315080035F00B205BE00C2059E0002057E0032055E043
S315080036000A2053E0012051E00D204FE00D204DE047
S315080036100D204BE00D2049E00D2047E00D2045E048
S315080036200D2043E00D2041E00D203FE00D203DE058
S315080036300D203BE00D2039E0012037E00D2035E074
S3150800364004287FF407AFF7E702366661E5612B4485
S3150800365023626B18A3626BE74FF0FF332361E360C5
S3150800366080232371BBE706F2FF16B7EB562FE5D387
S31508003670F2E74FF0FF332361E3608023237194F868
S31508003680612094F8603043EA02231BB2012B3FF411
S3150800369074AF0322A3E700BF9C0F002055AAFFFFC3
S315080036A05252614172724161980F002005B0BDE81F
S315080036B0F08300BF2DE9F04F83B0044689460768BA
S315080036C04FF0FF0A55460426D0464FF6FF7B7AE0B0
S315080036D03846FEF7EFFF0646002878D1E0690378FA
S315080036E0002B7ED0C27A02F03F02A271E52B5DD094
S315080036F02E2B5DD022F02001082914BF00210121BC
S31508003700494557D10F2A48D113F0400F06D090F8F3
S315080037100DA003F0BF032269626203E09D4218BF51
S3150800372045464AD190F80DE0D64545D1C17E827E00
S3150800373052EA01224ED1A26A11460192027802F09B
S315080037403F02013A02EB420602EB8606284D05F1D6
S315080037500D0A4FF0010C009363468C4615F8012BB1
S3150800376081184978825C42EA012233B1FE2E31D8AB
S315080037702CF816201346013601E05A452AD1AA45E7
S31508003780ECD1009B027812F0400F26D0FE2E21D8ED
S315080037900022019921F816201FE01DB9FEF700FF47
S315080037A0824520D04FF0FF3363621CE0454604E0B3
S315080037B0454602E0454600E0454600212046FFF71B
S315080037C09DFA064618B9A169002981D15EB1002380
S315080037D0A36108E0F2464546EFE7013BDDB2F24653
S315080037E0EBE70426F3E7304603B0BDE8F08F00BFE9
S315080037F0AC4C0008CA7E8B7E43EA02230278032A71
S3150800380005D1487D0A7D42EA002243EA024318466A
S31508003810704700BF2DE9F04F85B00546D0F80090F7
S31508003820884611F8013B2F2BFAD05C2BF8D00023E1
S31508003830AB6098F800301F2B08D82B6A8022DA7202
S3150800384000212846FFF746F903465CE14FF0010AD6
S31508003850AE6A98F800001F280DD92F280ED05C28CC
S315080038600FD0A6F1020B474601241AE02F280AD0EA
S315080038705C2811D107E00024534604E0002453468F
S3150800388001E0002453464344984613F8012B2F2A97
S31508003890FAD05C2AF8D01FE0B3F5807F00F02981C2
S315080038A01C46514600F0DAFD0146002800F0218149
S315080038B07F2809D8222800F0E880954A12F8013FA7
S315080038C013B19842FAD1E0E02BF8021F631C17F8EF
S315080038D0010F1F28CAD8D6E7202834BF0427002797
S315080038E0002C00F0F28006EB440232F8023D202B51
S315080038F001D02E2B03D1013CF7D1B346E6E0600098
S31508003900002326F81430002C00F0F3802B6A03F10C
S315080039100B01202203F8012B9942FBD1B11E00238B
S3150800392000E0013331F8022F202AFAD02E2AF8D0E7
S31508003930002B00F0CF8047F00307CBE0013C05D110
S315080039400822019200220292039204E032F8021D34
S315080039502E29F3D1F4E703F1010B36F813000028FA
S3150800396060D0202803D02E2805D1A34503D047F0E0
S3150800397003075B46EFE7029B019A934202D2A345EF
S3150800398019D1B8E0019B0B2B06D147F003072B6A28
S315080039901A78E52A56D14AE0A34502D047F003072C
S315080039A040D8039B9B00DBB2039323460B2201926C
S315080039B008220292CFE77F2840F29380002100F088
S315080039C04DFD0346002800F09B80524A134413F825
S315080039D0801C88B247F0020740B12B2906D04E4A10
S315080039E012F8013F002B7ED08B42F9D147F003072E
S315080039F05F200FE0039B43F0020303930AE0A0F164
S31508003A0061039BB2192B05D8039B43F0010303936B
S31508003A10203880B22B6A02990A4658545B4601320E
S31508003A20029298E72B6A1A78E52A04D101E00B225C
S31508003A30019205221A70019B082B03D1039B9B0058
S31508003A40DBB20393039A02F00C030C2B03D002F0AB
S31508003A500302032A01D147F0020717F0020F0AD121
S31508003A60039A02F00302012A08BF47F01007042B45
S31508003A7008BF47F008072B6ADF722846FFF7FEF9EA
S31508003A802B6ADA7A034660B101E006233BE0042894
S31508003A9039D102F00402D2B2002A14BF0346052324
S31508003AA031E012F0040F2ED1AB7913F0100F0AD0C3
S31508003AB02B69C3F3080303F1300149444846FFF76D
S31508003AC099FEA860C4E605231DE0B3460023ABF8BB
S31508003AD00030DAE702383218315A2E293FF430AF6F
S31508003AE02CE7014679E7A0F141039BB2192B81D94E
S31508003AF085E7062307E0019B0B2B7FF452AF44E7CB
S31508003B0047F0020772E7184605B0BDE8F08F00BF18
S31508003B10184C00082C4C0008244C000810B584B03A
S31508003B2001900091144604A840F8041DFEF748FDCC
S31508003B30002816DB114B53F820300BB100221A70FF
S31508003B40019BA3B100221A70019B0C4A42F820304F
S31508003B504BB1012C09D1002201A96846FFF70EFCDA
S31508003B600AE00B2008E0002006E0002004E000231D
S31508003B70024A42F82030184604B010BD9C0F0020B7
S31508003B802DE9F04393B00191002800F09C8004468B
S31508003B9015460023036002F01F06324606A901A84F
S31508003BA0FFF7ECFB002840F09080069B079303ABD9
S31508003BB00F935A4B1193019907A8FFF72BFE03465B
S31508003BC0002840F083800F9B93F90B30002B80F27E
S31508003BD088807FE0042B40F08C8007A8FFF72CFA3A
S31508003BE046F00806034650B193E09DF8223013F0DC
S31508003BF0110F40F0878015F0040F40F0858016F00D
S31508003C00080F46D00E9B00259D73DD73612119743C
S31508003C1048225A740E9B9D75DD7519765A762022B0
S31508003C200E9BDA72069FDDF8388041463846FFF764
S31508003C30E1FD81462A4641463846FEF759FE0E9B67
S31508003C401D775D779D77DD770122069BDA70B9F1DE
S31508003C50000F1CD0069BDD6A0022494607A8FFF71D
S31508003C6003F80346002854D129460698FEF722FD94
S31508003C7009F1FF33069AD36048B14BE015F0020FFD
S31508003C8002D013F0010F41D115F0080F01D046F00C
S31508003C902006069BDB6A23620E9B6362069D0E9FC7
S31508003CA039462846FFF7A6FDA06007F11C00FEF777
S31508003CB055FCE060002060746061E0612674256050
S31508003CC0EB88A38026E0092024E023E015F01C0FEA
S31508003CD00BD07FE715F01C0F18BF062309D1062362
S31508003CE003E015F01C0F80D106E0002BD6D018464D
S31508003CF010E046F00806F8E79DF8223013F0100F9A
S31508003D0006D1BBE7072005E0082003E0072300E00B
S31508003D100423184613B0BDE8F08300BF980D0020B1
S31508003D202DE9F04F85B00446884615461F46002300
S31508003D303B6003A9FEF770FC002840F0A280607C77
S31508003D40002840F0A280237C13F0010F00F09A802F
S31508003D50E36866699E1BAE4228BF2E46002E00F019
S31508003D60938004F1280301936369C3F30802002AC8
S31508003D706DD1039A5289013A12EA532912D10BB925
S31508003D80A06803E0A1692046FEF73AFE012802D89A
S31508003D900220607479E0B0F1FF3F02D1012060741F
S31508003DA073E0A061DDF80CA0A1695046FEF7ECFBB4
S31508003DB0054610B90220607467E04D445FEA562B49
S31508003DC024D0BAF80A3009EB0B029A4288BFC9EB2D
S31508003DD0030B5B462A4641469AF80100FCF798FD14
S31508003DE010B10120607450E0237C13F0400F0AD014
S31508003DF0E069401B834506D94FF40072019908EB28
S31508003E004020FEF7B7FB4FEA4B252EE0E2699542C4
S31508003E101CD0237C13F0400F0DD0012301999AF88A
S31508003E200100FCF7BBFD10B1012060742DE0237C76
S31508003E3023F04003237401232A4601990398407806
S31508003E40FCF766FD10B1012060741EE0E56161694A
S31508003E50C1F30801C1F50075B54228BF35462831BA
S31508003E602A4621444046FEF785FBA84463692B444D
S31508003E7063613B682B443B60761B7FF475AF00207B
S31508003E8003E002E0072000E0002005B0BDE8F08F5F
S31508003E902DE9F04F85B00446884616461F4600238E
S31508003EA03B6003A9FEF7B8FB002840F0BD80607CA4
S31508003EB0002840F0BB80237C13F0020F00F0B58089
S31508003EC06369F34228BFDE43002E00F0A78004F1A1
S31508003ED0280301936369C3F30802002A7DD1039A74
S31508003EE05289013A12EA53291DD133B9A06858B943
S31508003EF000212046FEF74CFE03E0A1692046FEF7A6
S31508003F0047FE002800F08A80012802D1022060744A
S31508003F108CE0B0F1FF3F02D10120607486E0A06119
S31508003F20A36803B9A060237C13F0400F0ED00123C9
S31508003F30E269019903984078FCF730FD10B1012039
S31508003F40607473E0237C23F040032374DDF80CA02F
S31508003F50A1695046FEF718FB054610B902206074A1
S31508003F6064E04D445FEA562B24D0BAF80A3009EBD0
S31508003F700B029A4288BFC9EB030B5B462A464146A9
S31508003F809AF80100FCF70AFD10B1012060744DE0B3
S31508003F90E169491B8B450AD94FF4007208EB4121A8
S31508003FA00198FEF7E7FA237C23F0400323744FEACF
S31508003FB04B2524E0E3699D420ED06269E3689A4284
S31508003FC00AD201232A4601999AF80100FCF7A0FCB7
S31508003FD010B10120607429E0E5616069C0F308004A
S31508003FE0C0F50075B54228BF354628302A464146F1
S31508003FF02044FEF7BFFA237C43F040032374A84409
S3150800400063692B446361E268934238BF1346E360F1
S315080040103B682B443B60761B7FF45CAF237C43F004
S3150800402020032374002001E000E0072005B0BDE866
S31508004030F08F00BF70B582B004460E460A2902D139
S315080040400D21FFF7F7FF6368002B14DB5D1C234483
S315080040501E733C2D0BDD01AB2A4604F10C012068CA
S31508004060FFF716FF019B5D1B18BF4FF0FF35656014
S31508004070A3680133A36002B070BD00BF30B583B03A
S31508004080044601A9FEF7C8FA00283ED1237C13F09E
S31508004090200F3BD013F0400F0CD00123E26904F146
S315080040A0280101984078FCF779FC88BB237C23F02B
S315080040B040032374216A0198FEF7FCFA50BB656A2F
S315080040C0EB7A43F02003EB72A26829462068FEF7D4
S315080040D00FFCE3682B771A0A6A771A0CAA771B0E65
S315080040E0EB770023AB75EB7561222A7648226A7650
S315080040F0AB74EB740122019BDA700198FEF7F6FAAD
S31508004100237C23F02003237404E003E0002001E06D
S315080041100120FFE703B030BD10B582B00446FFF7B3
S31508004120ADFF034638B901A92046FEF775FA0346DE
S3150800413008B900222260184602B010BD70B582B0D8
S3150800414004460D4601A9FEF767FA002840F0A88044
S31508004150607C002840F0A880E268AA4206D2237C48
S3150800416003F00203DBB2002B08BF15466369002281
S315080041706261002D00F09580019A568976026BB12E
S31508004180013B6A1EB2FBF6F2B3FBF6F18A4205D38F
S31508004190724213406361ED1AA16912E0A16879B908
S315080041A02046FEF7F5FC0146012802D1022060747C
S315080041B07AE0B0F1FF3F02D10120607474E0A0609C
S315080041C0A161002937D0B54225D9237C13F0020F07
S315080041D005D02046FEF7DCFC014620B91AE0204649
S315080041E0FEF70EFC0146B1F1FF3F02D101206074D3
S315080041F05AE0012903D9019B5B69994202D302203F
S31508004200607451E0A161636933446361AD1BAE42DA
S31508004210DBD300E0354663692B446361C5F30803C5
S315080042205BB10198FEF7B0F910B9022060743BE063
S3150800423000EB552502E0002500E000256369C3F37D
S31508004240080313B3E26995421FD0237C13F0400F8D
S315080042500ED0012304F1280101984078FCF79EFB53
S3150800426010B1012060741FE0237C23F040032374FF
S3150800427001232A4604F1280101984078FCF748FBF7
S3150800428010B1012060740FE0E5616369E26893424A
S3150800429009D9E360237C43F020032374002003E05C
S315080042A002E0002000E0002002B070BD30B591B0F9
S315080042B001900D46002205A901A8FFF75FF80446FC
S315080042C0A8B902AB0D930B4B0F93019905A8FFF7FD
S315080042D0A1FA044658B90D9B93F90B30002B05DB60
S315080042E02DB1294605A8FEF70FFB00E00624204657
S315080042F011B030BD980D002070B59CB00190022217
S3150800430005A901A8FFF73AF8059B1193034600286B
S3150800431048D102AB1993254B1B93019911A8FFF7B6
S3150800432079FA034600283DD1199B93F90B30002BE7
S3150800433035DB9DF84A4014F0010F32D11DE0069591
S315080043400896002106A8FEF7C5FB034650BB0021C8
S3150800435006A8FFF7AFF90346F8B1042816D021E0FE
S3150800436036B10022314611A8FEF77EFC0346C8B9CD
S315080043700598FEF7BBF9034614E0059D18992846EB
S31508004380FFF738FA064614F0100FD8D111A8FEF731
S3150800439049FD03460028E3D004E0072302E006238C
S315080043A000E0072318461CB070BD00BF980D00201A
S315080043B02DE9F04182B080461746054600244E1E78
S315080043C012E06B46012201A93846FFF7A9FC009BBB
S315080043D0012B0DD19DF804300D2B05D06A1C2B70CE
S315080043E001340A2B03D01546B442EADB00E0154631
S315080043F000232B709C4214BF4046184602B0BDE805
S31508004400F08100BF10B594B00446019100230293D1
S315080044100393017851B101A8FFF70CFE14F8011FA8
S315080044200029F8D1029A002A01DA0CE000226B462C
S3150800443004A90198FFF72CFD40B9009B029A9A42FD
S3150800444007D1039807E04FF0FF3004E04FF0FF3044
S3150800445001E04FF0FF3014B010BD00BF7F281BD914
S3150800446011B9C72808D112E0FF2814D8A0F1800393
S315080044700A4A32F813007047084A012332F8021F25
S31508004480814205D001339BB2802BF7D100E000238F
S315080044908033D8B270470020704700BF784D0008B7
S315080044A0F0B52449244BB0F5805F38BF1946074656
S315080044B004310C4631F8043C002B39D0984237D3E6
S315080044C031F8022C150AD2B2BE46D618B04229DAFD
S315080044D0082D2DD8DFE805F0050A101316191C1F3C
S315080044E02200C3EB070E31F81E00F0BDC31A03F015
S315080044F00103C01A80B2F0BD103880B2F0BD203872
S3150800450080B2F0BD303880B2F0BD1A3880B2F0BD46
S31508004510083080B2F0BD503880B2F0BDA0F5E35047
S3150800452080B2F0BD0431002DC3D104EB4201BFE7D0
S31508004530F0BD00BFBC4C0008784E0008034BFE22B5
S31508004540DA7018710222A3F844207047A00F0020E1
S31508004550054B00221A709A6483F84320A3F8442076
S315080045609A705A70704700BFA00F0020024B187847
S31508004570003018BF01207047A00F00200022024B10
S3150800458083F84320704700BFA00F002038B5037892
S31508004590FF2B22D1FDF7AEFC18B91020FFF7CEFF8E
S315080045A061E1AD4C0023637001252570FF22E2709E
S315080045B0102222716371FDF7E7FBA071FDF7F6FB88
S315080045C0E071FDF7F3FB000A20726572A5720823F5
S315080045D0A4F84430FDF730FA45E104469E4A1278BD
S315080045E0012A40F06081C93B352B00F23981DFE8AA
S315080045F013F0C000370137012F01370137012601B3
S31508004600DB0015010501370137013701370137018D
S3150800461037013701370137013701370137013701CC
S3150800462037013701370137013701370137013701BC
S3150800463037013701370137013701370137013701AC
S315080046403701370137017600510036006D00370112
S315080046503701370192003701A400A800B600457853
S31508004660FDF792FB0138854203DD2220FFF766FF3E
S31508004670F9E0794D6278A96C281DFCF795FFFF23B0
S31508004680EB706378AA6C1344AB6463780133A5F8BE
S315080046904430E8E04578FDF777FB0138854203DDCD
S315080046A02220FFF74BFFDEE061686B4DA964627854
S315080046B0281DFCF779FFFF23EB706378AA6C134477
S315080046C0AB6463780133A5F84430CCE0624BFF2233
S315080046D0DA7042689A640122A3F84420DDE05E4B52
S315080046E0FF22DA709A6C406840B11044002312F831
S315080046F0011B0B44DBB29042F9D100E00023564A75
S31508004700C2F80730012313710023537193710823EC
S31508004710A2F84430C1E0504BFF22DA704F4A9A643F
S3150800472000221A715A719A710721D9711A725A722E
S315080047309A720822A3F84420AFE00020FFF7FEFE95
S3150800474091E0454BFF22DA7000221A7159785971A7
S315080047509A71DA711A720622A3F844209DE03E4B3C
S3150800476000221A705A70FF22DA700122A3F8442038
S3150800477093E0394B9D6CFDF707FB621C411E2846EA
S31508004780FDF75EF918B93120FFF7D8FE6BE0324C19
S31508004790FF23E370FDF7F8FA0138A36C0344A3641A
S315080047A00123A4F8443078E04578FDF7EDFA02389D
S315080047B0854203DD2220FFF7C1FE54E0264BFF2287
S315080047C0DA700122A3F84420617839B9FDF748F96F
S315080047D0002848D13120FFF7B1FE44E0A21C1E4B49
S315080047E0986CFDF72DF918B93120FFF7A7FE3AE0C6
S315080047F0194A6378916C0B44936434E0164CFF2392
S31508004800E370002525716571FDF7BEFAA071E571A3
S31508004810257265720723A4F844303EE041680E4BC2
S31508004820986CFDF711F918B93120FFF787FE1AE0E1
S31508004830094BFF22DA700122A3F844202DE0FCF789
S3150800484097FE054BFF22DA700122A3F8442024E0E4
S315080048503120FFF773FE06E0A00F00206C50000819
S315080048602020FFF76BFE104B93F84330012B02D143
S315080048701020FFF763FE0C4BB3F94410002912DD34
S315080048800948012380F8433089B20330FDF766FAF8
S3150800489038BD054BB3F94410F2E7034B93F84330A0
S315080048A0012BF6D1E4E738BDA00F002008B5074B69
S315080048B0044613B10021AFF30080054B1868836ADC
S315080048C003B19847204600F033F800BF0000000007
S315080048D0785100080E4B70B51E460E4C0025E41A9A
S315080048E0A410A54204D056F8253098470135F8E7B4
S315080048F000F020F8084B094C1E46E41AA4100025BF
S31508004900A54204D056F8253098470135F8E770BD1A
S315080049107C0000207C0000207C0000208000002015
S3150800492003460244934202D003F8011BFAE7704794
S31508004930FEE70000F8B500BFF8BC08BC9E46704705
S31508004940F8B500BFF8BC08BC9E4670472F64656D75
S315080049506F70726F675F73746D3332663230372EDD
S3150800496073726563000000002F626F6F746C6F6767
S315080049702E747874000000002E2E5C2E2E5C2E2ECF
S315080049805C2E2E5C536F757263655C41524D434DC8
S31508004990335F53544D333246325C63616E2E630087
S315080049A005020602060307030803090309040A04A5
S315080049B00B040C040C050D050E050F050F06100655
S315080049C01007100800000800100018002000280032
S315080049D030003800400048005000580000800008A9
S315080049E0004000000200000000C00008004000006F
S315080049F00300000000000108000001000400000098
S31508004A00000002080000020005000000000004087B
S31508004A100000020006000000000006080000020070
S31508004A20070000002E2E5C2E2E5C2E2E5C2E2E5C91
S31508004A30536F757263655C41524D434D335F5354F2
S31508004A404D333246325C756172742E630000000085
S31508004A50303A00002E2E5C2E2E5C2E2E5C2E2E5CFE
S31508004A60536F757263655C66696C652E630000003A
S31508004A704669726D77617265207570646174652028
S31508004A8072657175657374206465746563746564AD
S31508004A900A0D00004F70656E696E67206669726D53
S31508004AA0776172652066696C6520666F722072652B
S31508004AB06164696E672E2E2E000000004552524F23
S31508004AC0520A0D004F4B0A0D000000005374617224
S31508004AD074696E67207468652070726F6772616D9D
S31508004AE06D696E672073657175656E63650A0D007D
S31508004AF050617273696E67206669726D7761726557
S31508004B002066696C6520746F20646574656374201B
S31508004B10657261736520626C6F636B732E2E2E004F
S31508004B2045726173696E672000000000206279741F
S31508004B3065732066726F6D206D656D6F7279206181
S31508004B40742030780000000052656164696E672041
S31508004B506C696E652066726F6D2066696C652E2EAF
S31508004B602E4552524F520A0D00000000496E7661DA
S31508004B706C696420636865636B73756D20666F7511
S31508004B806E642E2E2E4552524F520A0D000000001A
S31508004B9050726F6772616D6D696E67200000000064
S31508004BA020627974657320746F206D656D6F7279F4
S31508004BB0206174203078000057726974696E672026
S31508004BC070726F6772616D20636865636B73756D6C
S31508004BD02E2E2E00436C6F73696E67206669726DA0
S31508004BE0776172652066696C650A0D004669726DA3
S31508004BF07761726520757064617465207375636387
S31508004C0065737366756C6C7920636F6D706C65740B
S31508004C1065640A0D00000000222A3A3C3E3F7C7F6C
S31508004C20000000002B2C3B3D5B5D0000809A45414F
S31508004C308E418F804545454949498E8F9092924FBE
S31508004C40994F555559999A9B9C9D9E9F41494F55F9
S31508004C50A5A5A6A7A8A9AAABACADAEAFB0B1B2B38D
S31508004C60B4B5B6B7B8B9BABBBCBDBEBFC0C1C2C37E
S31508004C70C4C5C6C7C8C9CACBCCCDCECFD0D1D2D36E
S31508004C80D4D5D6D7D8D9DADBDCDDDEDFE0E1E2E35E
S31508004C90E4E5E6E7E8E9EAEBECEDEEEFF0F1F2F34E
S31508004CA0F4F5F6F7F8F9FAFBFCFDFEFF0103050734
S31508004CB0090E10121416181C1E0000007D1D010096
S31508004CC0632C001E9601A01E5A01001F0806101F1D
S31508004CD00606201F0806301F0806401F0606511F35
S31508004CE00700591F521F5B1F541F5D1F561F5F1F6A
S31508004CF0601F0806701F0E00BA1FBB1FC81FC91FFA
S31508004D00CA1FCB1FDA1FDB1FF81FF91FEA1FEB1F8D
S31508004D10FA1FFB1F801F0806901F0806A01F08061B
S31508004D20B01F0400B81FB91FB21FBC1FCC1F01005B
S31508004D30C31FD01F0206E01F0206E51F0100EC1F75
S31508004D40F21F0100FC1F4E210100322170211002C2
S31508004D50842101008321D0241A05302C2F04602CCD
S31508004D600201672C0601752C0201802C6401002DB6
S31508004D70260841FF1A030000C700FC00E900E2000C
S31508004D80E400E000E500E700EA00EB00E800EF00D9
S31508004D90EE00EC00C400C500C900E600C600F40039
S31508004DA0F600F200FB00F900FF00D600DC00A200C6
S31508004DB0A300A500A7209201E100ED00F300FA0088
S31508004DC0F100D100AA00BA00BF001023AC00BD0054
S31508004DD0BC00A100AB00BB009125922593250225B6
S31508004DE024256125622556255525632551255725F0
S31508004DF05D255C255B251025142534252C251C25C9
S31508004E0000253C255E255F255A25542569256625F6
S31508004E10602550256C25672568256425652559254F
S31508004E205825522553256B256A2518250C258825CE
S31508004E3084258C2590258025B103DF009303C003C4
S31508004E40A303C303B500C403A6039803A903B403C5
S31508004E501E22C603B50329226122B10065226422F7
S31508004E6020232123F7004822B0001922B7001A226E
S31508004E707F20B200A025A00061001A03E0001703F6
S31508004E80F8000703FF000100780100013001320134
S31508004E900601390110014A012E0179010601800136
S31508004EA04D00430281018201820184018401860149
S31508004EB08701870189018A018B018B018D018E018A
S31508004EC08F0190019101910193019401F6019601D8
S31508004ED09701980198013D029B019C019D012002C2
S31508004EE09F01A001A001A201A201A401A401A6019B
S31508004EF0A701A701A901AA01AB01AC01AC01AE014A
S31508004F00AF01AF01B101B201B301B301B501B501FA
S31508004F10B701B801B801BA01BB01BC01BC01BE01A9
S31508004F20F701C001C101C201C301C401C501C40121
S31508004F30C701C801C701CA01CB01CA01CD011001C9
S31508004F40DD0101008E01DE011201F3010300F1010A
S31508004F50F401F401F8012801220212013A020900BB
S31508004F60652C3B023B023D02662C3F024002410291
S31508004F70410246020A015302400081018601550298
S31508004F8089018A0158028F015A0290015C025D026A
S31508004F905E025F0293016102620294016402650285
S31508004FA066026702970196016A02622C6C026D021C
S31508004FB06E029C01700271029D01730274029F01C8
S31508004FC076027702780279027A027B027C02642CE6
S31508004FD07E027F02A60181028202A901840285025D
S31508004FE086028702AE014402B101B20145028D0272
S31508004FF08E028F0290029102B7017B030300FD0324
S31508005000FE03FF03AC0304008603880389038A03AF
S31508005010B1031103C2030200A303A303C4030803D5
S31508005020CC0303008C038E038F03D8031801F20305
S315080050300A00F903F303F403F503F603F703F7038A
S31508005040F903FA03FA033004200350041007600436
S3150800505022018A043601C1040E01CF040100C004EE
S31508005060D004440161052604000000004F70656EF7
S31508005070424C5400002020202020202020202828D0
S3150800508028282820202020202020202020202020FA
S31508005090202020202088101010101010101010103A
S315080050A0101010101004040404040404040404106A
S315080050B010101010101041414141414101010101F8
S315080050C001010101010101010101010101010101C2
S315080050D010101010101042424242424202020202CE
S315080050E00202020202020202020202020202020292
S315080050F01010101020000000000000000000000042
S315080051000000000000000000000000000000000091
S315080051100000000000000000000000000000000081
S315080051200000000000000000000000000000000071
S315080051300000000000000000000000000000000061
S315080051400000000000000000000000000000000051
S315080051500000000000000000000000000000000041
S315080051600000000000000000000000000000000031
S3150800517000000000004300001C00002000000000A2
S30D0800518060B0FF7F010000008A
S3150800518801000000000000000102030401020304F4
S31508005198060708090400000074500008000000000B
S315080051A800000000000000000000000000000000E9
S315080051B8000000000000000000000000755100080B
S315080051C800000000000000000000000000000000C9
S315080051D800000000000000000000000000000000B9
S315080051E800000000000000000000000000000000A9
S315080051F8000000000000000000000000A9010008E7
S309080052088501000806
S70508000000F2
